:1000000009C025C00DC00CC00BC00AC009C008C083
:1000100007C006C011241FBECFE9CDBF47D0A6C080
:10002000EFCF86B1806C86B93699FECF84B185B1A9
:10003000379890E06EE170E087D09C0128513C4FEA
:10004000C9010895EEDFC09A62D0C09808951F924A
:100050000F920FB60F9211242F933F934F935F93FC
:100060006F937F938F939F93AF93BF93EF93FF9380
:100070008FEF9DEEA2E081509040A040E1F700C0DC
:100080000000B19902C0C39ADDDFFF91EF91BF91EB
:10009000AF919F918F917F916F915F914F913F9120
:1000A0002F910F900FBE0F901F901895F89487B363
:1000B000896087BBC19A8BB780648BBF85B782602C
:1000C00085BF17B887B1826687B97894C098C39AFC
:1000D0008FEF9DEEA2E081509040A040E1F700C07C
:1000E0000000C3988FEF91EFABE281509040A040A9
:1000F000E1F700C00000EACF07C0EFE5F9E0319773
:10010000F1F700C0000081508823B9F7089507C0B7
:10011000EFE5F9E03197F1F700C000000197009793
:10012000B9F7089505C093E09A95F1F70000815062
:100130008823C9F7089505C023E02A95F1F7000048
:1001400001970097C9F708955527002480FF02C042
:10015000060E571F660F771F6115710521F09695E2
:100160008795009799F7952F802D0895F894FFCFE4
:00000001FF
